:100000000C94E8030C9420040C9420040C94200419
:100010000C9420040C9420040C9420040C942004D0
:100020000C9420040C9420040C9420040C94CF27EE
:100030000C947E280C947A220C9420040C942004B6
:100040000C9420040C9420040C9420040C9402239F
:100050000C9420040C9420040C9420040C94200490
:100060000C9420040C9420040C9420040C94200480
:100070000C942004C207C207EE07EE076309630968
:10008000630963095608EF0800090009EB281229E3
:100090000A2A12290A2A5E2981290A2AD829E72947
:1000A0001E001F0020002100220000002300240069
:1000B00025002600270000000000000000000000CE
:1000C0000000280044454255473A20646973616244
:1000D0006C65642E0A0044454255473A20656E61BE
:1000E000626C65642E0A000A0025303258006C6587
:1000F000645F7461736B3A20004F6E6573686F7450
:100100003A206163746976653A2025640A000A0022
:1001100025303862003A200025303258000A722F0C
:10012000632030313233343536370A007267626CFF
:10013000696768742074696D6572206469736162AF
:100140006C652E0A007267626C6967687420746956
:100150006D657220656E61626C65642E0A0072675F
:10016000626C696768742073657420687376205BBD
:100170004E4F454550524F4D5D3A2025752C257503
:100180002C25750A007267626C6967687420736554
:100190007420687376205B454550524F4D5D3A2080
:1001A00025752C25752C25750A007267626C6967A8
:1001B0006874207261696E626F772073657420685D
:1001C00073763A2025642C25642C25642C25750A29
:1001D000007267626C696768742064697361626C3D
:1001E00065205B454550524F4D5D3A207267626C09
:1001F000696768745F636F6E6669672E656E6162BA
:100200006C65203D2025750A007267626C6967681D
:100210007420656E61626C65205B454550524F4DA0
:100220005D3A207267626C696768745F636F6E66BF
:1002300069672E656E61626C65203D2025750A0038
:100240007267626C6967687420746F67676C652099
:100250005B454550524F4D5D3A207267626C69674D
:1002600068745F636F6E6669672E656E61626C6548
:10027000203D2025750A007267626C6967687420EA
:100280006D6F6465205B4E4F454550524F4D5D3A52
:100290002025750A007267626C69676874206D6F4B
:1002A0006465205B454550524F4D5D3A2025750AE7
:1002B000007267626C696768745F696E6974207246
:1002C00067626C696768745F636F6E6669672E6DDD
:1002D0006F6465203D20302E20577269746520645C
:1002E000656661756C742076616C75657320746FDA
:1002F00020454550524F4D2E0A007267626C696767
:1003000068745F696E6974206565636F6E6669679E
:10031000206973206E6F7420656E61626C65642E57
:100320000A007267626C696768745F696E6974203D
:100330007374617274210A007267626C6967687411
:100340005F696E69742063616C6C65642E0A00726B
:1003500067626C696768745F636F6E6669672E7346
:1003600070656564203D2025640A007267626C69CF
:100370006768745F636F6E6669672E76616C203D97
:100380002025640A007267626C696768745F636F36
:100390006E6669672E736174203D2025640A0072C1
:1003A00067626C696768745F636F6E6669672E6801
:1003B0007565203D2025640A007267686C6967686E
:1003C000745F636F6E6669672E6D6F6465203D2094
:1003D00025640A007267626C696768745F636F6E98
:1003E0006669672E656E61626C65203D2025640A32
:1003F000007267626C696768745F636F6E666967D5
:1004000020454550524F4D3A0A0000047F3F1F647B
:100410003214643214783C1E1E140A052223252649
:1004200028292A2C2D2F3032333536383A3B3D3EA1
:100430004042434547494A4C4E5051535557595AEB
:100440005C5E6062646668696B6D6F717375777905
:100450007B7D7F81838587898A8C8E909294969804
:100460009A9C9E9FA1A3A5A7A8AAACAEAFB1B3B416
:10047000B6B8B9BBBCBEBFC1C2C3C5C6C7C9CACB6B
:10048000CCCDCED0D1D2D2D3D4D5D6D7D7D8D9D936
:10049000DADADBDBDBDCDCDCDCDCDDDDDDDDDCDC9F
:1004A000DCDCDCDBDBDBDADAD9D9D8D7D7D6D5D4BC
:1004B000D3D2D2D1D0CECDCCCBCAC9C7C6C5C3C288
:1004C000C1BFBEBCBBB9B8B6B4B3B1AFAEACAAA8DD
:1004D000A7A5A3A19F9E9C9A98969492908E8C8A91
:1004E00089878583817F7D7B79777573716F6D6B6C
:1004F0006968666462605E5C5A5957555351504E44
:100500004C4A4947454342403E3D3B3A38363533F5
:1005100032302F2D2C2A292826252322FFAA7F5569
:100520004000010101010101010101020202020278
:10053000020202020303030303030303040404048B
:100540000404040505050505060606060607070753
:10055000070708080808090909090A0A0A0B0B0B0A
:100560000C0C0C0D0D0D0E0E0E0F0F0F10101111A7
:10057000111212131314141515161617171818192B
:10058000191A1A1B1B1C1D1D1E1E1F202021222292
:10059000232424252626272829292A2B2C2D2D2ED5
:1005A0002F30313232333435363738393A3B3C3DEF
:1005B0003E3F404142434445464748494A4C4D4EE0
:1005C0004F50515354555658595A5B5D5E5F6162A6
:1005D00064656668696B6C6D6F7072737577787A35
:1005E0007B7D7E8082838587888A8C8E8F91939590
:1005F00096989A9C9EA0A2A3A5A7A9ABADAFB1B3B4
:10060000B5B7BABCBEC0C2C4C6C9CBCDCFD1D4D693
:10061000D8DBDDDFE2E4E7E9EBEEF0F3F5F8FAFD35
:10062000FF0A002530325820006B6579626F6172D5
:10063000645F7265706F72743A200064656C5F6B02
:1006400065795F6269743A2063616E27742064651E
:100650006C3A20253032580A006164645F6B65791A
:100660005F6269743A2063616E2774206164643A42
:1006700020253032580A005B735D005B575D005BDC
:10068000535D005B525D001003470054004D002095
:1006900000500061006400000026035300700061F8
:1006A000006300650043006900740079004B006539
:1006B00000790062006F0061007200640073000046
:1006C000000403090409025B00030100A0FA090405
:1006D0000000010301010009211101000122400075
:1006E000070581030800010904010001030000005F
:1006F000092111010001223B0007058203200001AE
:100700000904020002030000000921110100012276
:1007100022000705830320000107050303200001D1
:100720001201000200000008EDFE906002000102CC
:1007300000010631FF0974A1010975150026FF00AB
:100740009520750881020976150026FF0095207511
:10075000089102C005010906A1018506050719E0F7
:1007600029E7150025019508750181020507190083
:1007700029EF1500250195F0750181020508190181
:100780002905950575019102950175039101C00533
:10079000010906A101050719E029E71500250195C2
:1007A0000875018102950175088101050719002965
:1007B000FF150026FF009506750881000508190140
:1007C0002905950575019102950175039101C000F8
:1007D00011241FBECFEFD4E0DEBFCDBF04B603FEB1
:1007E00018C08091860290918702A0918802B091F2
:1007F00089028730904BA740B04B59F41092860283
:10080000109287021092880210928902E0E0F8E3C9
:10081000099511E0A0E0B1E0E0E6F6E502C0059040
:100820000D92A237B107D9F722E0A2E7B1E001C0EB
:100830001D92A638B207E1F70E947A150C942E2B70
:100840000C940000FF93EF93E0917201F09173011B
:10085000309709F00995EF91FF910895FC0185917A
:10086000803011F0EFDFFBCF0895FF27E0E230E2A8
:1008700047FF0CC0419597FF09C0EDE26095709568
:1008800080959095611D711D811D911D27FF02C0EE
:10089000219530E350E2AA27660F771F881F991F22
:1008A000AA1FA41710F0A41B63955A95A9F7AA30A4
:1008B00008F0A95FA05DAF93F395611571058105FF
:1008C000910541F7ED3211F4EF93F395F21718F417
:1008D0003F93F395FBCF8F91B5DFFA95E1F708953C
:1008E000E991F9918591803021F0853219F0AADFE4
:1008F000F9CF089520E0E89455915532C1F3503373
:1009000011F4689455915A3348F4505390F3220FE0
:10091000022E220F220F200D250FF4CF0EF4219569
:1009200089919991533619F3533729F1533559F178
:10093000BC0188279927E8945C3621F48991999124
:1009400068945591543639F446EF7EF077FF0DC028
:100950008FEF9FEF0AC055374AE039F0583540E134
:1009600021F0523642E009F00895FF93EF937DDFC6
:10097000EF91FF91B7CFFF93EF93FC01819180300E
:10098000B9F360DFFBCFFF93EF9368DFF1CFDF9325
:10099000CF93CDB7DEB72596A3DFCF91DF91089532
:1009A0008091180286608160809318020895662302
:1009B00011F08BE401C08EE40E94700781E008957D
:1009C00081E0089581E008950C94E20408950C9468
:1009D000E6041F93CF93DF9300D000D01F92CDB7D2
:1009E000DEB749835A836B833091750189819A817F
:1009F000311114C0662359F0222349F00E949D0B47
:100A0000182F682F89819A810E943D0B03C00E9494
:100A10006E0B182F69817A81812F04C00E949D0B73
:100A200069817A810F900F900F900F900F90DF9156
:100A3000CF911F910C94BD12FC01262F4081518152
:100A40006281738184810C94E90481E00895CF93DD
:100A5000DF93EC0160E00E941C05BE01DF91CF91A5
:100A60000C94E7040C9449140C94471408950E94C4
:100A7000E7090E9436052FEF84E39CE02150804077
:100A80009040E1F700C000000C9428230F931F93BF
:100A9000CF93DF938C0161E00E941C05EC01B8014B
:100AA0000E94E404882309F462C0B801CE010E94C8
:100AB0007720882309F45BC0B801CE010E942C1E68
:100AC000882309F454C0B801CE010E94D31F8823A3
:100AD00009F44DC0B801CE010E94321D882309F4EB
:100AE00046C0F80182818823D9F1CF3D8CE5D80733
:100AF00079F140F4C115FCE5DF0791F0C130DC4528
:100B000091F02EC0CC35EDE5DE0741F1CD35FDE5A8
:100B1000DF0709F1CB35DD4519F50E94301020C003
:100B20000E94370524C080911802C82FC095C1705B
:100B3000C0FB80F980931802CC2329F086ED90E069
:100B40000E942E0414C084EC90E00E942E0410C079
:100B50000E94E4100CC00E94271002C00E943310B3
:100B6000C801DF91CF911F910F910C94E004C0E078
:100B70008C2FDF91CF911F910F9108950E945D22DC
:100B80000C94E9050E94EC050C9463228295982F41
:100B90009373292F220F220F982F9C7C9695969560
:100BA000922B892F8575880F9A7A9695892B0895AF
:100BB00008950C94D80581E008950C94DB05089500
:100BC000CF93C82F0E94D9058C2F0E94DD05CF91AD
:100BD000089580E00C94E0050E94D3200C94E00579
:100BE000CF930E94D320C82F80917401C81741F180
:100BF000C09374018091180282FF1EC080FF04C060
:100C00008EEE90E00E942E048091180280FF0CC0AE
:100C10001F92CF9389EE90E09F938F930E94C70419
:100C20000F900F900F900F908091180280FF04C0DA
:100C300087EE90E00E942E048C2FCF910C94E0055B
:100C4000CF910895CF93DF93CDB7DEB72B970FB633
:100C5000F894DEBF0FBECDBF4F83588769877A8770
:100C60008B8761110E945F0F9E012F5F3F4F86E0CF
:100C7000F90111928A95E9F785E0FE013796D901CD
:100C800001900D928A95E1F789819A814C815D816D
:100C9000452B31F09F3F31F491E08F3F19F403C0B1
:100CA00091E001C090E090FF09C049815A816B81B9
:100CB0007C818D819E810E947B0E05C0C9010E94AE
:100CC00025058111F2CF2B960FB6F894DEBF0FBE2B
:100CD000CDBFDF91CF910895FC01808191810E9469
:100CE000DF0B0895CF93882309F482C0C82F823880
:100CF000C1F40E94D32081FD7BC069E38091020191
:100D0000909103010E9418220E94810F2FEF81EE23
:100D100094E0215080409040E1F700C0000069E37A
:100D200019C08338F1F40E94D32080FD61C063E5CF
:100D300080910201909103010E9418220E94810F6C
:100D40002FEF81EE94E0215080409040E1F700C009
:100D5000000063E580910201909103010E9423222B
:100D600044C08438C1F40E94D32082FD41C067E4AE
:100D700080910201909103010E9418220E94810F2C
:100D80002FEF81EE94E0215080409040E1F700C0C9
:100D9000000067E4DFCF8CEF8C0F813AD0F46C2F2A
:100DA00080910201909103010E947621882349F0ED
:100DB0006C2F80910201909103010E9423220E94D6
:100DC000810F6C2F80910201909103010E941822E3
:100DD0000CC080E28C0F883058F4C77081E001C0ED
:100DE000880FCA95EAF70E94420FCF910C94810FA9
:100DF000CF910895882309F45BC0682F823879F475
:100E00000E94D32081FF54C069E380910201909138
:100E100003010E9418220E94810F69E310C08338E9
:100E2000B1F40E94D32080FF43C063E580910201AA
:100E3000909103010E9418220E94810F63E5809126
:100E40000201909103010E9423220C94810F8438A7
:100E500079F40E94D32082FF2BC067E480910201C5
:100E6000909103010E9418220E94810F67E4E7CF4E
:100E70008CEF860F813A18F380E2860F883048F4B1
:100E8000677081E001C0880F6A95EAF70E94480FF9
:100E9000DCCF8BE5860F833020F480E090E00C946B
:100EA0003421685A673120F480E090E00C944A21A4
:100EB00008951F93CF93DF93182FEB010E947206C2
:100EC000209741F08FE99FE00197F1F700C0000003
:100ED0002197F6CF812FDF91CF911F910C94FA06C5
:100EE000893319F060E070E002C060E570E00C94B6
:100EF0005907882321F00E94420F0C94810F089516
:100F0000882321F00E94480F0C94810F0895CF92FE
:100F1000DF92EF92FF920F931F93CF93DF937C01A9
:100F2000D62FC72FFC011281058102950F700E94F8
:100F3000380F8823B9F01123A9F08C2F807F8034DB
:100F400021F080E28D0F883068F080915D0282FD93
:100F500009C082E00E94E10F0E94380F91E0D82E74
:100F6000D92601C0D12CCC2EC2948FE0C8228C2D62
:100F700090E08C30910508F0A6C1FC01E65CFF4FC3
:100F80000C94C62A8C2F807FCF70882311F0C295D5
:100F9000C07F112399F0CC2309F481C180E28D0F29
:100FA000883010F0D11104C08C2F0E94420F03C072
:100FB0008C2F0E94520F0E94810F71C18D2F0E94B1
:100FC000FA06CC2309F47FC180E28D0F883038F116
:100FD000DD2329F18C2F0E94580F24C08C2F807F95
:100FE000CF70803211F0C295C07FDD2319F0D1306F
:100FF000A1F13DC080915D0282FF17C0112349F02D
:10100000CC2329F08C2F0E94420F0E94810F80E098
:1010100047C180E00E94FA06CC2309F454C18C2F0A
:101020000E94480F0E94810F4EC1112371F00023CE
:1010300041F0013031F40E94620F8C2B0E946A0F44
:1010400042C10E94620F8C2B1DC0002319F0013099
:1010500009F439C10E94770F25C0112321F0063011
:1010600008F031C10EC0053008F02DC11BC011239E
:1010700061F0002331F0F701858180FF10C18F708E
:1010800085838C2F0E9479071EC1002359F0D93324
:1010900009F016C1FFEF07EE13E0F15000401040D9
:1010A000E1F70CC18C2F0E9480070DC18C2F83703B
:1010B00009F047C011110BC12D2F229526952770DD
:1010C000220F220F6D2F6F70862F90E0A0E0B0E00E
:1010D000022E04C0880F991FAA1FBB1F0A94D2F7C3
:1010E000D4FF10C04FE050E060E070E004C0440F57
:1010F000551F661F771F2A95D2F74095509560952A
:10110000709503C040E050E0BA01C695C695C37023
:101110008A019B01082B192B2A2B3B2BC901B801F3
:10112000C23049F058F4C13019F00E94530ACFC0C0
:101130000E94410ACCC00E94650AC9C00E943F0AB1
:10114000C6C0112319F08C2F817001C086958823A9
:1011500009F4BDC02D2F229526952770220F220F4E
:101160006D2F6F70862F90E0A0E0B0E0022E04C0DB
:10117000880F991FAA1FBB1F0A94D2F7D4FF10C073
:101180004FE050E060E070E004C0440F551F661F60
:10119000771F2A95D2F7409550956095709503C0BA
:1011A00040E050E0BA01C695C695C3708A019B0124
:1011B000082B192B2A2B3B2BC901B801C23049F04F
:1011C00058F4C13019F00E94180B81C00E94060B20
:1011D0007EC00E942A0B7BC00E94790A78C0CF7023
:1011E000112339F08C2F0E949F0A8D2F0E947907BE
:1011F0006EC08D2F0E9480078C2F0E94C00A67C08E
:10120000D23F21F128F4D03F41F0D13FC1F043C09B
:10121000D33F19F1D43F79F03EC0112341F005309E
:1012200008F051C08C2F8F710E94E50A4CC0063027
:1012300008F049C0F7CF80915D0282FF18C01123EA
:1012400039F08C2F8F710E949F0A3DC01123C9F382
:101250008C2F8F710E94C00A36C0112329F08C2F69
:101260008F710E948A0A2FC00E94850A2CC0112308
:1012700049F0CF718C2F0E949F0A63E08C2F0E944F
:10128000C60F21C081E00E94E10F0230E0F082E051
:101290000E94E10F18C0112331F0002391F28D2F2D
:1012A0000E94720610C0002399F2D93349F41FEF4F
:1012B00027EE33E0115020403040E1F700C000003D
:1012C0008D2F0E94FA0688EF8C0D843020F40E9446
:1012D000D3200E94E005DD20C9F00E94340F80FD7C
:1012E00015C0F70112820E942E0F0E949F0AC701AB
:1012F0000E94A7090E942E0FDF91CF911F910F919D
:10130000FF90EF90DF90CF900C94C00ADF91CF91C7
:101310001F910F91FF90EF90DF90CF9008950F9362
:101320001F93CF93DF93EC01688179818A810E94BA
:10133000EA0B8C010E943C0B0E942D0AB801CE01E1
:101340000E948707DF91CF911F910F910895CF934E
:10135000DF93EC01988189812B813C81232B31F033
:101360008F3F31F481E09F3F19F403C081E001C059
:1013700080E080FD1DC0CE010E944605811110C095
:101380000E94380F8823A1F08A81882389F08091F8
:101390005D0282FD0DC082E0DF91CF910C94E10FE0
:1013A000CE010E948F09CE01DF91CF910C942705C9
:1013B000DF91CF9108950E945F0F0C94810F80916F
:1013C0000201909103010E942E220C94DB090E94DD
:1013D0004F0F0C94DF0992959F70963079F010F4BE
:1013E000925001C09A50923068F4803F69F018F42E
:1013F000883E40F409C0843F29F406C0883E20F0AE
:10140000813F11F080E0089581E00895FC01808122
:1014100091810E94DF0B0E94EB090895CF93DF9327
:1014200000D000D01F92CDB7DEB70F900F900F9075
:101430000F900F90DF91CF910895CF93DF9300D05D
:1014400000D000D0CDB7DEB726960FB6F894DEBF39
:101450000FBECDBFDF91CF910895089508950C94EC
:101460002E0A0C942F0A0E94310A6093890170930E
:101470008A0180938B0190938C010C94DB090C946E
:10148000330A0F931F930091890110918A012091D3
:101490008B0130918C01602B712B822B932B1F9130
:1014A0000F910C94330A0F931F93009189011091AF
:1014B0008A0120918B0130918C016023712382235A
:1014C00093231F910F910C94330A0F931F93009154
:1014D000890110918A0120918B0130918C01602744
:1014E0007127822793271F910F910C94330A0C9434
:1014F0002E0A0E94770A609385017093860180937B
:101500008701909388010C94DB0960E070E0CB01C7
:101510000C94790A0F931F9341E050E060E070E073
:101520008A019B0104C0000F111F221F331F8A95DF
:10153000D2F7C901B8011F910F910C94790A0F934A
:101540001F9341E050E060E070E004C0440F551F7D
:10155000661F771F8A95D2F7809185019091860149
:10156000A0918701B09188018A019B01082B192B5A
:101570002A2B3B2BC901B8011F910F910C94790ABA
:101580000F931F9341E050E060E070E004C0440F0F
:10159000551F661F771F8A95D2F740955095609525
:1015A00070958091850190918601A0918701B091FD
:1015B00088018A019B01082319232A233B23C9019F
:1015C000B8011F910F910C94790A0F931F9341E07A
:1015D00050E060E070E004C0440F551F661F771FA5
:1015E0008A95D2F78091850190918601A09187011B
:1015F000B09188018A019B01082719272A273B27D8
:10160000C901B8011F910F910C94790A0F931F9390
:101610000091850110918601209187013091880108
:10162000602B712B822B932B1F910F910C94790AB5
:101630000F931F93009185011091860120918701DE
:101640003091880160237123822393231F910F918E
:101650000C94790A0F931F930091850110918601D4
:101660002091870130918801602771278227932775
:101670001F910F910C94790A0895282F362F892FE6
:1016800066E00E943D2A820F982F9770A1E001C06A
:10169000AA0F9A95EAF786958695869590E065E07B
:1016A00070E00E94462AFC01EA58FE4F40E050E0FC
:1016B000632F70E090819B01042E02C03695279520
:1016C0000A94E2F72170219529272A2329272193BB
:1016D0004F5F5F4F4530510569F70895282F892FD7
:1016E00066E00E943D2A820FA82FA77086958695F6
:1016F000869590E065E070E00E94462ABC0140E0DB
:1017000050E080E0FB01E40FF51FEA58FE4F208116
:1017100030E00A2E02C0369527950A94E2F7217030
:101720003327042E01C0220F0A94EAF7822B4F5F61
:101730005F4F4530510531F70895BF92CF92DF9248
:10174000EF92FF920F931F93CF93DF938C01C09082
:101750008501D0908601E0908701F090880180910A
:10176000890190918A01A0918B01B0918C01C82AC6
:10177000D92AEA2AFB2ACFE1D0E0D701C6010C2EF4
:1017800004C0B695A795979587950A94D2F780FDE2
:1017900004C0219790F7B12C07C0BC2EB8018C2F44
:1017A0000E94D8120197A9F38B2DDF91CF911F9141
:1017B0000F91FF90EF90DF90CF90BF900895CF935F
:1017C000DF93EC010E949D0BBE010E94D812DF91B5
:1017D000CF9108951F93CF93DF93EB019091750103
:1017E000992321F0CB010E94DF0B13C0882349F01D
:1017F000CB010E949D0B182F682FCE010E943D0B3C
:1018000004C0CB010E946E0B182FBE01812F0E94D5
:10181000D812DF91CF911F910895CF93DF93C0919C
:101820008D0180918E01C817A1F0D0E0CE0166E055
:1018300070E00E94462AFC01E157FE4F4081518131
:1018400062817381848195810E941D0A2196C770EF
:10185000E8CFDF91CF9108954091BF015091C00131
:101860006091C1017091C2018091C3019091C40146
:101870000C941D0AFF920F931F93CF93DF938091D7
:10188000C40182958F7009F062C08091C1018823E4
:1018900009F45DC020918D01F0908E011091BF017F
:1018A0000091C001A091C201B091C30181E01F3F2E
:1018B00009F080E0C0910001D0910101482F2F155F
:1018C00009F445C0109721F00F3F21F080E003C0DC
:1018D00081E001C0842F30E080FD35C0C90166E0A1
:1018E00070E00E94462AFC01E157FE4F818180137F
:1018F0002AC08081811327C08281811124C0838105
:1019000094818A1B9B0B8C179D07E8F48091C4017E
:101910008F7080618093C401C90166E070E00E940D
:10192000462AFC01EC56FE4F90819F709061908397
:101930008FEB91E00E94A709DF91CF911F910F914A
:10194000FF900C940D0C2F5F3F4F2770B8CFDF91A5
:10195000CF911F910F91FF9008959F92AF92BF92E8
:10196000CF92DF92EF92FF920F931F93CF93DF936B
:10197000CDB7DEB761970FB6F894DEBF0FBECDBF0F
:101980008C0185E0F801DE011D9601900D928A958B
:10199000E1F7F801E2809091BF013091C0016091C0
:1019A000C2017091C3016115710531F03F3F31F4FF
:1019B00081E09F3F19F403C081E001C080E0F82F6F
:1019C000F1709F2E80FD47C1F80140812181A380E5
:1019D000B4808FEBC82E81E0D82EF090C101F501C4
:1019E000E61BF70B6091000170910101FF2009F4E3
:1019F000DCC08091C401582F507FE617F70708F02C
:101A000096C0511155C0231313C0491311C0FE2CA9
:101A1000E1100EC08F7080618093C4010E942C0C75
:101A2000C6010E94A7098091C401F801858350C1B5
:101A3000AB2831F02F3F31F481E04F3F19F403C060
:101A400081E001C080E080FD03C081E08E2502C0FE
:101A500080E090E0F82FF170FF2E80FF1FC0E09132
:101A60008D0130918E01E31709F410C1F0E0CF0130
:101A700066E070E00E94462ADC01A157BE4F119635
:101A80008C911197281307C08C91481304C01296AB
:101A90008C91E81203C03196E770E5CFFE2CEE2062
:101AA00009F416C18091C40181608093C40154C0BF
:101AB000231306C0491304C0E11002C0F80199C005
:101AC000C8010E94060A882361F1EE2051F120919D
:101AD000C401822F82958F7090E0029774F08091FC
:101AE000BF019091C00198878F831986BB86AA8613
:101AF0002C87CE0107960E94A70986E0F801AFEB7C
:101B0000B1E001900D928A95E1F70E943A0C0E9493
:101B10002C0C0AC0231711F1C8010E94060A81117A
:101B20002CC0C8010E94A709FF24F394D1C0511111
:101B3000F1CF7A2DB98AA88A522F6E2D89890E94F9
:101B40000E0A8FEB91E00E94A70986E0F601119240
:101B50008A95E9F70E942C0CF12CBAC04913DCCF0E
:101B6000E110DACFF8018583C8010E94A70986E059
:101B7000F60111928A95E9F7ABC0EE2091F220911F
:101B8000C401822F82958F7090E002970CF4B5CF3C
:101B90008091BF019091C0019A8389831B82BD828D
:101BA000AC822E83CE010196A6CFE617F70708F088
:101BB00044C0FE2CEE2009F4B4CF231330C04913E7
:101BC0002EC02091C40120FD21C0822F82958F70EC
:101BD000482F50E041155105C9F0F80125834F30D9
:101BE000510541F08F5F982F9295907F822F8F70D3
:101BF000892B8583C8010E94A70986E0F801AFEB15
:101C0000B1E001900D928A95E1F73DC086E0F801C0
:101C1000AFEBB1E001900D928A95E1F759C0C80190
:101C20000E94060A811169CF8091C401816080936E
:101C3000C401C8010E94A7094BC07A2DB98AA88A9D
:101C4000522F6E2D89890E940E0A86E0F6011192AC
:101C50008A95E9F718C0EE2009F463CFC8010E9405
:101C6000060AF82E882309F45CCF86E0F801AFEB72
:101C7000B1E001900D928A95E1F78FEB91E00E941F
:101C80006C060E943A0C0E942C0C22C04D872E87B5
:101C90008D859E850E94DF0B292F22952F70223083
:101CA00028F49F7039F0811105C00BC0243028F44E
:101CB0009F7049F4805E883020F0C8010E94A70917
:101CC0009F2CF92C05C0F8019581907F99F7F9CFE9
:101CD0008F2D61960FB6F894DEBF0FBECDBFDF919A
:101CE000CF911F910F91FF90EF90DF90CF90BF9019
:101CF000AF909F900895CF93DF93CDB7DEB72C9729
:101D00000FB6F894DEBF0FBECDBF4F8358876987EB
:101D10007A878B879C87CE0107960E94AD0C88231B
:101D2000D1F09F8188852A853B85232B31F08F3F19
:101D300031F481E09F3F19F403C081E001C080E0ED
:101D400080FD6FC04F81588569857A858B859C851C
:101D50000E941D0A66C086E0FE013796DE011196DC
:101D600001900D928A95E1F7FF81E8856A857B8570
:101D70006115710531F0EF3F31F481E0FF3F19F457
:101D800003C081E001C080E080FD4BC080918E01E6
:101D900090E09C012F5F3F4F2770332740918D01CA
:101DA00050E02417350709F443C0F983EA837D83A3
:101DB0006C8366E070E00E94462ADC01A157BE4FAA
:101DC00096E0FE01319601900D929A95E1F72093ED
:101DD0008E010E940D0C25C090E066E070E00E942C
:101DE000462A81579E4F0E94AD0C882371F1809145
:101DF0008D0190E066E070E00E94462AFC01E15708
:101E0000FE4F4081518162817381848195810E945E
:101E10001D0A80918D0190E001968770992780932B
:101E20008D0180918D0190918E018913D5CF0DC0C8
:101E30000E94E70910928E0110928D01EFEBF1E004
:101E400086E0DF011D928A95E9F72C960FB6F8948B
:101E5000DEBF0FBECDBFDF91CF9108958091E50128
:101E600085958595859508958091E50187700895FC
:101E70009091E501977081E009F480E008958091E8
:101E80000802089590910802892B80930802089512
:101E900080959091080289238093080208951092FA
:101EA0000802089590910702892B809307020895F4
:101EB00080959091070289238093070208951092DC
:101EC000070208958091E601089508950C94650F26
:101ED0000C94660F90915D0292FD08C09091E6010E
:101EE000981721F08093E6010C94680F0895809173
:101EF000E601882329F01092E60180E00C94680F37
:101F00000895CF93DF93E0910201F0910301809156
:101F100008028083E0910201F09103019081809199
:101F20000702892B80838091E601882381F0E0916C
:101F30000201F09103019081892B8083809102013D
:101F4000909103010E94602181110E94770FC0913E
:101F50000201D091030140E250E065EC71E0CE0156
:101F60000E94D92A892B69F080E2FE01A5ECB1E03C
:101F700001900D928A95E1F7CE01DF91CF910C94FB
:101F8000DF20DF91CF9108950C94650F90915D0251
:101F900092FD10C0982F990F990F990F692B60939C
:101FA000E5010E949F0A8091E501859585958595BB
:101FB0000C94C40F0C949F0A1092E50180E00C94DD
:101FC000C40F2091E501809582238093E501982F2D
:101FD000977099F430E0482F082E000C550B241709
:101FE000350759F090915D0292FD07C08595859562
:101FF00085950E94C00A0C94DC0F0895CF939091B0
:102000005D0292FB222720F92817F9F0C82F892FAB
:10201000C0FB82F980935D0280915C0290915D0229
:102020000E94601082E00E94E10F8091180280FF00
:102030000CC01F92CF9389EF90E09F938F930E94E3
:10204000C7040F900F900F900F90CF91089580913B
:102050005D0282FB882780F991E089270C94FE0FAE
:1020600081E00C94FE0F80E00C94FE0F6FEF7FEF89
:1020700080E090E00C94182B80E090E00E94F42A1D
:1020800021E0893E9E4F09F020E0822F089582E0F2
:1020900090E00C94E62A83E090E00C94E62ACF933B
:1020A00084E090E00E94E62AC82F82E290E00E943D
:1020B000E62A2C2F30E0A901582BCA01CF910895B0
:1020C000CF93C92F682F84E090E00E94FA2A6C2FEA
:1020D00082E290E0CF910C94FA2AAB01BC018FE030
:1020E00090E00C940C2BAB01BC0183E190E00C94CC
:1020F0000C2B60E070E0CB010C94731060E070E09A
:10210000CB010E946D100C94791069EE7EEF80E097
:1021100090E00E94182B60E082E090E00E94FA2A92
:1021200060E083E090E00E94FA2A10928901109208
:102130008A0110928B0110928C0160E084E090E0A3
:102140000E94FA2A60E082E290E00E94FA2A60E0AF
:1021500085E090E00E94FA2A60E086E090E00E942C
:10216000FA2A6FEF87E090E00E94FA2A40E050E000
:10217000BA0188E090E00E940C2B60E08DE090E0D6
:102180000E94FA2A40E050E0BA0188E190E00E9403
:102190000C2B60E087E190E00E94FA2A40E050E0DA
:1021A000BA018CE190E00E940C2B60E070E080E2CC
:1021B00090E00E94182B40E050E0BA0188E190E0E6
:1021C0000E940C2B0C947E100C948510682F8EE0CE
:1021D00090E00C94FA2A0E94E72260931402709314
:1021E0001502809316029093170260931002709369
:1021F0001102809312029093130208950E94E72225
:102200006093140270931502809316029093170244
:1022100060930C0270930D0280930E0290930F0254
:10222000089581E008950C94111108950C941511EE
:102230000C9415110C9418110C9415110C941C117C
:102240000C94151188EC94E20E94C9200E94201180
:102250000C941E110E9416110C9415110E94CC139F
:102260000C94DF050E94D2220E94DF140E942E11DE
:102270000E94D51B0E947D1F0C941A118F929F9271
:10228000AF92BF92CF92DF92EF92FF920F931F9384
:10229000CF93DF93CDB7DEB72A970FB6F894DEBFA2
:1022A0000FBECDBF0E94F414982E81110E94EB1036
:1022B00089E0A82E82E0B82E00E010E0802E802F6A
:1022C0000E94F013D82EF501C1905F01C826B1F429
:1022D0000F5F1F4F0330110589F78FEF89838A83C2
:1022E0001B820E94DB228160782F9D838C83498131
:1022F0005A816B818D810E9422062FC08091180225
:1023000081FD0E94F613E12CFF24F3948C2D8F2184
:10231000F1F00E941311882399F0EE828F82DF2062
:1023200081E009F480E088870E94DB228160782FB9
:102330009A8789874E815F8168858A850E942206F7
:10234000F801E75FFD4F8081F826F08206C0E39434
:10235000FF0CF6E0EF12DACFBBCF81E0911001C0A5
:1023600080E02A960FB6F894DEBF0FBECDBFDF9196
:10237000CF911F910F91FF90EF90DF90CF90BF9082
:10238000AF909F908F9008950E943E110E94841CF0
:102390000E94901F81110E94FE100C94F005CF93B3
:1023A000DF930E94DD12EC01811523E59207A0F571
:1023B000811532E5930708F0A2C0811540E2940729
:1023C000C0F4811551E0950708F0D3C0853A910516
:1023D00050F48430910508F0CCC0019709F0C6C0D4
:1023E00081E090E0C7C0805E9109089708F4C1C001
:1023F000BDC0C11581E5D80708F07BC0C11520E537
:10240000D20708F052C0C11530E4D30708F4AEC0BB
:10241000DF70CE01906AAEC0811546E5940708F5DD
:10242000811555E5950708F087C0C11584E5D807E3
:1024300008F07CC09E012370332781E090E002C049
:10244000880F991F2A95E2F7C695C695D0E065E0FA
:10245000CC0FDD1F6A95E1F7C82BD92BCE019A6806
:1024600089C081152AE5920780F4811539E5930723
:1024700008F06BC0811548E5940708F477C0D82FA1
:10248000CC27CE01806F906A75C09056811590421E
:1024900008F06CC08D2F8F710E947113DD27D06200
:1024A0008F71AE01582BCA0165C0CE01F4E096953C
:1024B0008795FA95E1F7282F23703C2F337081E040
:1024C00090E002C0880F991F3A95E2F79C68AC0132
:1024D000522B9C2F9F7096959695892F90E0EC013A
:1024E000A5E0CC0FDD1FAA95E1F7CA018C2B9D2B2F
:1024F00041C0DC2FCC27CE01816F906A3BC09C018C
:102500002370332781E090E002C0880F991F2A953D
:10251000E2F7C695C695D0E075E0CC0FDD1F7A9541
:10252000E1F7C82BD92BCE019C6824C0DC2FCC2727
:10253000CE01846F906A1EC00E9471138F7190E06B
:10254000D82FCC27CE01906215C08F700E947113D6
:1025500094E0D695C7959A95E1F7CF70D0E0DC2F3F
:10256000CC27D0699E01282BC90104C080E090E0EF
:1025700001C0CE01DF91CF910895382F262F872FEC
:1025800090E066E070E00E94462AFC01832F90E014
:1025900062E170E00E94462A8E0F9F1FFC01E20F4D
:1025A000F11DEE0FFF1FE056FF4F859194910895A6
:1025B0000E94BD120E94CF1108958238910569F1E1
:1025C000B0F48133910509F46DC048F48932910566
:1025D00009F463C08A32910509F469C0089585330E
:1025E000910509F455C089339105B9F00895833EEA
:1025F000910569F138F4803E9105B1F0823E910574
:1026000009F10895863E9105A9F1873E9105B9F13A
:10261000843E910509F064C023C020915C0220FD36
:102620004FC021FD4DC0089580915C0280FD44C0E3
:1026300080915D0280FF44C080915C0284FD42C0B5
:1026400083EE4DC080915C0282FF38C0F5CF80914F
:102650005C0282FD33C080915D0280FD31C0ECCF11
:1026600080915D0281FF32C080915C0284FD2AC0AE
:1026700087EE35C080915C0283FF26C0F5CF809144
:102680005C0283FD21C080915D0281FD1FC0ECCF03
:1026900080915C0285FD1CC01DC080915C0285FD9F
:1026A00019C016C080915C0286FD16C017C08091CB
:1026B0005C0286FD13C010C089E311C082EE0FC01A
:1026C00080EE0DC080E00BC086EE09C084EE07C02E
:1026D00089E205C085E303C08AE201C081E390E09E
:1026E000089590915C0292FF0DC0282F2871283028
:1026F00019F4877F846006C0282F2471243011F4D8
:102700008B7F886093FF0DC0282F2871283119F422
:10271000877E846106C0282F2471243111F48B7EBA
:10272000886120915D0220FF0DC0382F387138304C
:1027300019F4877F816006C0382F3171313011F470
:102740008E7F886021FF0DC0282F2871283119F451
:10275000877E816106C0282F2171213111F48E7E80
:10276000886194FD877E08950C9436100E94F414BD
:102770008FE39CE90197F1F700C000000E94F41478
:1027800080E00E94F01380FF04C00E94B4130C94F8
:10279000282308950C94B6130E943C10811102C0A6
:1027A0000E94E4100E944710809318020E944F106C
:1027B00090935D0280935C020E94CA130E944B10AA
:1027C000682F70E080E090E00E943F0A60918501F0
:1027D0007091860180918701909188010C94770A0D
:1027E000E82FF0E0EF59FD4F80810895CF92DF92FE
:1027F000EF92FF920F931F93CF93DF938DE191E0C0
:102800000E942E0481E6E82E82E0F82EC0E0D0E09F
:1028100098E1C92E91E0D92E00E111E0DF93CF932A
:10282000DF92CF920E94C70485E191E00E942E04BE
:10283000F70181917F010E94C6051F928F931F931C
:102840000F930E94C7048EE091E00E942E0421960F
:102850008DB79EB708960FB6F8949EBF0FBE8DBF7A
:10286000C330D105D9F6DF91CF911F910F91FF9021
:10287000EF90DF90CF90089580EA8A95F1F7089560
:1028800000C008950C943C1408950C9444140C94C6
:1028900045140C94D004F894E82FE295EF70F0E022
:1028A00031A1282F2F7081E090E001C0880F2A9578
:1028B000EAF7982F9095932391A392A1892B82A355
:1028C00078940895CF93DF9384E60E944B1485E6B5
:1028D0000E944B1481E90E944B14C4E2D1E089911B
:1028E0008F3F11F00E944B1481E0CA32D807B9F72C
:1028F000DF91CF910895CF92DF92EF92FF920F93E5
:102900001F93CF93DF938C01C62FD0E0CE01865D5D
:102910009E4F7C01FC0190819F3F09F447C0D62E59
:10292000F894E92FE295EF70F0E081A19F7021E02B
:1029300030E001C0220F9A95EAF7822B81A382A191
:102940002095282322A378940E944014E4E2F1E029
:102950004AE251E031E0C12C21912F3F89F0A22FB2
:10296000A295AF70B0E090968C9190E02F7002C06D
:10297000959587952A95E2F780FD02C0832F01C0C7
:1029800080E0C82A330F4E175F0731F7F7018081C7
:102990008F3F11F00E944B1461E0C11001C060E054
:1029A0008D2D0E944214C00FD11FC882DF91CF919C
:1029B0001F910F91FF90EF90DF90CF9008950E94AC
:1029C000621483E0E1E6F2E0DF01982F1D929A9510
:1029D000E9F7EEE5F2E0DF011D928A95E9F783E081
:1029E0000E9437150C9432051F93CF93DF9300D0CC
:1029F0001F92CDB7DEB719821A821B8260E0CE012A
:102A000001960E947B1461E0CE0101960E947B1426
:102A100062E0CE0101960E947B1443E050E0BE01CB
:102A20006F5F7F4F8EE592E00E94D92A11E00097F8
:102A300009F410E0892B49F089819A81AB81809358
:102A40005E0290935F02A0936002212F43E061E653
:102A500072E08EE592E00E9438150E943405812FC5
:102A60000F900F900F90DF91CF911F9108950895CF
:102A7000FF920F931F93CF93DF938C01F62ED72FE6
:102A8000C42F222349F081E080931B020E94DB22A5
:102A900090931A028093190280911B028823C1F03F
:102AA0008091190290911A020E94F322059780F0FA
:102AB000EF2DFD2FD8014C2F50E0CD01801B910B45
:102AC000841795071CF48D918193F7CF10921B0208
:102AD000DF91CF911F910F91FF9008950E9444259F
:102AE0000E9432110C9450250E9454250E94C4115A
:102AF0000C9472250E9479220E942B250E9422119B
:102B00000E946E150E9474150E942A11FBCFEF924D
:102B1000FF920F931F93CF93DF93E82F71110AC099
:102B2000442321F0F0E0EF5DFA4FE4916E2F7E2F09
:102B30008E2F6CC0C62FD0E0072F10E0282F30E07A
:102B4000442329F0F901EF5DFA4F249130E0CE01E2
:102B500066E070E00E94462AEE24EA94F12CB70168
:102B60000E947C2ADB01CC0FDD1FCB016BEA7FEFDB
:102B70000E94462A8C0F9D1FC82FCC0FC80FC7017B
:102B8000801B910BB9010E94462AE92F492FD0E002
:102B9000CE01B8010E94462A692F70E0C701861B4A
:102BA000970BB9010E94462AF92FC7018C1B9D0B78
:102BB000B8010E94462A692F70E0C701861B970B57
:102BC000B9010E94462AA230B10591F038F410975D
:102BD00059F01197C1F48E2F7F2F0CC0A430B1058E
:102BE00079F050F0169779F4722F842FE92F0DC0E9
:102BF000892F7E2FE22F09C0822F7E2FEF2F05C055
:102C0000822F792F02C0722F8F2F6E2FDF91CF91DD
:102C10001F910F91FF90EF90089541E00E9487155A
:102C2000089508950E940D160895CF93DF93762F8F
:102C3000E901682F842F0E941216798368838A83A2
:102C4000DF91CF91089580916402282F269530E07E
:102C50002115310519F48170826005C025323105D6
:102C600024F08170886480936402089588E090E085
:102C70000C94EE2ACF92DF92EF92FF926B017C01CF
:102C80000E942316B701A60188E090E0FF90EF9024
:102C9000DF90CF900C940C2BE4E6F2E083E080838D
:102CA00011828FEF8283838314826081718182819C
:102CB00093810C943A168091180280FF08C081EF2E
:102CC00093E09F938F930E94C7040F900F90809181
:102CD000180280FF0FC08091640281701F928F9351
:102CE00084ED93E09F938F930E94C7040F900F9001
:102CF0000F900F908091180280FF0FC080916402A6
:102D000086951F928F9389EB93E09F938F930E94F8
:102D1000C7040F900F900F900F908091180280FFC2
:102D20000EC0809165021F928F938FE993E09F936D
:102D30008F930E94C7040F900F900F900F90809177
:102D4000180280FF0EC0809166021F928F9385E863
:102D500093E09F938F930E94C7040F900F900F9062
:102D60000F908091180280FF0EC0809167021F9221
:102D70008F938BE693E09F938F930E94C7040F90ED
:102D80000F900F900F908091180280FF0EC08091DD
:102D900068021F928F938FE493E09F938F930E941A
:102DA000C7040F900F900F900F90089580916402C8
:102DB00080FF02C08695089580E008959091680292
:102DC000933018F49F5F90936802882351F06091CC
:102DD00064027091650280916602909167020C9482
:102DE0003A16089581E00C94DE16909168029923BA
:102DF00019F0915090936802882351F06091640219
:102E00007091650280916602909167020C943A1667
:102E1000089581E00C94F51670E00C94011E309139
:102E200008018091640280FF0CC08091070190E04E
:102E300063E070E00E94462A632F87599D4F0C94EF
:102E40000C172091090140910A01241770F7822F75
:102E500090E063E070E00E94462AFC01E759FD4FD4
:102E60001182108212822F5FF0CFA82FB62F80918F
:102E7000640280FF16C02091090130910A012317D6
:102E800070F4822F90E063E070E00E94462AFC011B
:102E9000E759FD4FA183B08342832F5FF0CF0C949D
:102EA0000F170895CF93DF9300D01F92CDB7DEB7F1
:102EB0009091640290FF0AC09E012F5F3F4F0E94D5
:102EC00015164B8169818A810E9435170F900F90EA
:102ED0000F90DF91CF910895CF93DF93EC01EC81B8
:102EE000F0E0E45EFB4F4491E4E6F2E06281818130
:102EF0000E9452178C818F5F8C83DF91CF91089550
:102F0000CF93DF93EC01E4E6F2E0438162818C81B0
:102F10000E9452178C818F5F8C83DF91CF9108952F
:102F20000F931F93CF93DF9300D01F92CDB7DEB7DF
:102F30008C0180911C0281110AC09E012F5F3F4FBE
:102F40004FEF6FEF0E9415168A8180931C02F801E3
:102F50008481813051F028F0823061F440911C026C
:102F60000AC080911C0240E007C060911C0240E052
:102F700080E003C040E080E060E00E943517F80187
:102F8000848190E0019663E070E00E94902A84833F
:102F90000F900F900F90DF91CF911F910F91089597
:102FA0004F925F926F927F928F929F92AF92BF9259
:102FB000CF92DF92EF92FF920F931F93CF93DF9305
:102FC00000D01F92CDB7DEB7182FD62E042F622E59
:102FD0009091640290FFB3C0E92FE695AE2FB0E068
:102FE000A35DBE4F8C91809326029E7F923061F448
:102FF0009E012F5F3F4F812F0E9415164B816981E3
:103000008A810E94351761C0823019F400916702ED
:103010005CC0863019F41091650257C08930D9F32D
:10302000893109F052C0E9512E2F2170722E81E0B2
:10303000C22EC826E695F0E0E45EFA4FE590F490E3
:10304000412CFF248AEAA82E81E0B82E20910B01A2
:103050004216C8F5842C912CC401B7010E94462A5F
:10306000622F70E00E947C2A512E711002C0560E11
:1030700001C0561A8091180280FF11C0FF92EF9292
:103080001F92CF921F925F921F924F92BF92AF9268
:103090000E94C7040FB6F894DEBF0FBECDBF80916B
:1030A00009019401280F311DC90163E070E00E94FD
:1030B000462A9C0127593D4F402F6D2D852D0E949A
:1030C00015164394C3CF0E940F1710936502D09238
:1030D0006602009367026620E9F0609164027091D5
:1030E000650280916602909167020E943A16809173
:1030F000180280FF24C0809167021F928F938091F5
:1031000066021F928F93809165021F928F9385E8CC
:1031100091E00CC08091180280FF11C01F920F93A4
:103120001F92DF921F921F938EE591E09F938F93E2
:103130000E94C7040FB6F894DEBF0FBECDBF0F903C
:103140000F900F90DF91CF911F910F91FF90EF9013
:10315000DF90CF90BF90AF909F908F907F906F90B7
:103160005F904F900895E4E6F2E09181282F43812B
:10317000628188E0890F0C94D01781E00C94B31819
:10318000E4E6F2E09181282F4381628188EF890F84
:103190000C94D01781E00C94C018E4E6F2E0628150
:1031A00021E1620F08F46FEF282F438181810C9495
:1031B000D01781E00C94CD18E4E6F2E0628121E1C1
:1031C000621B08F460E0282F438181810C94D017A2
:1031D00081E00C94DC18E4E6F2E0438121E1420F47
:1031E00008F44FEF282F628181810C94D01781E081
:1031F0000C94EB18E4E6F2E0438121E1421B08F471
:1032000040E0282F628181810C94D01781E00C94DA
:10321000FA1820E00C94D017EF92FF921F93CF93EF
:10322000DF93EC0110E0EE24EA94F12C30910B01D5
:10323000131700F520910901812F90E0820F911D55
:1032400063E070E00E94462AFC01E759FD4F632FBE
:1032500070E0C7010E94902A812F0E943D2A9C8124
:103260009F014091670260916602890F0E941516C6
:103270001F5FDCCF0E940F179A818C8190FF02C0E4
:103280008F5F01C081508C83DF91CF911F91FF90A0
:10329000EF900895BF92CF92DF92EF92FF920F933B
:1032A0001F93CF93DF93FC01828180FF02C0DFEF89
:1032B00001C0D1E0C0E080910B01C81708F040C008
:1032C00080910901CC2ED12C9601280F311DC90106
:1032D00063E070E00E94462A87599D4F7C01FC0103
:1032E00011821082128204E010E0B12C80911E0243
:1032F0008B0D853014F0837005C087FF03C090915B
:103300000B01890F082E000C990BC816D90691F4F1
:103310008091670290E0B8010E94462A95958795B2
:10332000959587959701482F609166028091650277
:103330000E941516BD0E01501109C1F6CF5FBBCF1B
:103340000E940F1780911E02D13031F4811102C00A
:1033500080910B01815007C090E0019660910B01B4
:1033600070E00E94902A80931E02DF91CF911F91FE
:103370000F91FF90EF90DF90CF90BF900895CF9383
:103380002091090130910A01231770F4822F90E0F7
:1033900063E070E00E94462AFC01E759FD4F11826C
:1033A000108212822F5FF0CFC0E060910B01C61730
:1033B00090F5EC2FF0E070E0CF010E94902A909100
:1033C0000901890F20911D02022E000C330B90E0A1
:1033D00063E070E00E94462AE217F307A4F0209110
:1033E0000601022E000C330B2E173F0764F09C01E0
:1033F00027593D4F409167026091660280916502B6
:103400000E94151606C0FC01E759FD4F118210827B
:103410001282CF5FCACF0E940F17209105018091C1
:103420001D02820F80931D0290910601920F9093CE
:10343000060119165CF4082E000C990B40910B0143
:1034400050E041505109841795071CF021952093B5
:103450000501CF9108954F925F926F927F928F9264
:103460009F92AF92BF92CF92DF92EF92FF920F9313
:103470001F93CF93DF938C01FC01C481CC2ED12C00
:10348000E12CF12CA7019601C701B6010E94572A31
:10349000A70196010E94572A4B015C0180E290E04F
:1034A0006C01CC1AD1080D2C000CEE08FF0825E5A4
:1034B00030E040E050E0C501B4010E94572A2B01E2
:1034C0003C01A7019601C701B6010E94572AA70136
:1034D00096010E94572A9B01AC01280D391D4A1DF7
:1034E0005B1DC301B2010E94A42AD22F822F90E05B
:1034F0002A3230F025E530E0A901481B590BCA01FA
:1035000063E070E00E94462A97FD019695958795A5
:10351000C82FC095F12C85E5E82EED1A80910B019E
:10352000F816D0F4F1FC02C0EE2D01C0ED2F209171
:1035300009018F2D90E0820F911D63E070E00E94E1
:10354000462A9C0127593D4F4C2F609166028E2FD1
:103550000E941516F394E2CF0E940F17F8018481A0
:10356000811102C091E003C0803219F49FEF909363
:10357000040190910401890FF8018483DF91CF91B8
:103580001F910F91FF90EF90DF90CF90BF90AF9081
:103590009F908F907F906F905F904F9008950F93C2
:1035A0001F93CF93DF93EC0100E010E040910B01FB
:1035B000842F90E0081719072CF5809109019801D4
:1035C000280F311DC90163E070E00E94462A9C016A
:1035D00027593D4F469550E08C81041715071CF480
:1035E000882331F002C0811103C04091670201C0FD
:1035F00040E060916602809165020E9415160F5F9F
:103600001F4FD4CF0E940F178C8190E001968170DC
:1036100099278C83DF91CF911F910F91089560912D
:103620006402669570E04BE050E08CE091E00E940F
:10363000CC2A892B19F481E0809327020E94DB2297
:103640009093200280931F028091180280FF08C08F
:1036500085E491E09F938F930E94C7040F900F9091
:103660000895109227028091180280FF08C08CE212
:1036700091E09F938F930E94C7040F900F9008953D
:103680009091640290FF54C09170811102C09260C9
:1036900006C0853210F0986402C0880F982B909372
:1036A00064026623B1F060916402709165028091BA
:1036B0006602909167020E943A168091180280FF7C
:1036C0001BC08091640286951F928F9385E992E0DA
:1036D0000BC08091180280FF0FC080916402869514
:1036E0001F928F9387E792E09F938F930E94C70466
:1036F0000F900F900F900F9060916402669570E0AC
:103700004BE050E08CE091E00E94CC2A892B19F02C
:103710000E94311B02C00E940F1B81E08093220295
:103720004091670260916602809165020C940919CC
:103730000895682F90916402969581E0890F8532F3
:1037400008F081E00C94401B81E00C94991B682FD9
:103750009091640296958FEF890F09F484E20C949E
:10376000401B81E00C94A71B61E00C94401B8091EE
:1037700064028160809364028091180280FF0DC012
:103780001F9281E08F9389E092E09F938F930E9434
:10379000C7040F900F900F900F9080916402869550
:1037A0000C94B41B60E00C94401B809125028111A5
:1037B00060C08091180280FF08C088E393E09F9367
:1037C0008F930E94C7040F900F908091180280FF82
:1037D00008C082E293E09F938F930E94C7040F90EA
:1037E0000F900E943C10811110C08091180280FF40
:1037F00008C08AEF92E09F938F930E94C7040F90B6
:103800000F900E94E4100E944C160E94361660939E
:1038100064027093650280936602909367026E7FE4
:10382000C1F48091180280FF08C081EB92E09F9361
:103830008F930E94C7040F900F900E944C160E9415
:1038400036166093640270936502809366029093CB
:1038500067020E9423160E945B1610922702809135
:10386000640280FF03C086950E94D21B81E0809392
:1038700025020895809164028E7F80936402609196
:1038800064027091650280916602909167020E94C5
:103890003A168091180280FF0FC0809164028170F7
:1038A0001F928F9381ED91E09F938F930E94C704A5
:1038B0000F900F900F900F900E94311B2FEF80E719
:1038C00092E0215080409040E1F700C000000C944D
:1038D0000F178091180280FF10C0809164028095BC
:1038E00081701F928F9380E492E09F938F930E9448
:1038F000C7040F900F900F900F908091640280FD8D
:103900000C943A1C0C94B71B0F931F93CF93DF9327
:1039100080912702882309F485C080912602E091D6
:103920006402E695E81BE0932102823049F4F0E05E
:10393000E85EFB4FE491CE2FD0E00CE617E149C0E2
:10394000863049F4F0E0EB5EFB4FE491CE2FD0E0FF
:1039500000E817E13EC0893051F4E695F0E0EE5EF4
:10396000FB4FE491CE2FD0E00CE019E132C08F3054
:1039700051F4E695F0E0E15FFB4FE491CE2FD0E00B
:103980000AE419E126C0853149F4F0E0E45FFB4F19
:10399000E491CE2FD0E00FEB19E11BC0883181F00C
:1039A000833239F4EAE0F4E0C591D49100E917E1FB
:1039B00010C0843251F4C4EFD1E00FEC1AE109C019
:1039C000C8E2D0E00BE21AE104C0C0EDD7E001E1AB
:1039D00016E180912202882361F0109222020E9457
:1039E000DB229093200280931F02109224021092F7
:1039F00023020E94DB22E0911F02F09120028E1B25
:103A00009F0B8F3F9F4770F4EC0FFD1FF093200238
:103A1000E0931F028FE192E0F801DF91CF911F91B7
:103A20000F910994DF91CF911F910F9108958823F1
:103A300011F0FA0101C0FB010994CF93DF93C82F65
:103A4000D62F0E94D6168C1740F00E94D6168D17DE
:103A500020F4DF91CF910C94A41B8C2FDF91CF9198
:103A60000C94B41B1F93CF93DF93FB0112811111B0
:103A7000C3C0EC010E943F0F8272CD3CFCE5DF0722
:103A800009F49AC0A8F5C73CECE5DE0709F476C056
:103A9000A8F4C43C9CE5D90709F45FC028F4C33CF2
:103AA000DC4509F457C054C0C53C9CE5D90709F46E
:103AB00059C0C63CDC4509F45CC04AC0CA3CFCE5C0
:103AC000DF0709F46AC050F4C83CECE5DE0709F4EE
:103AD0005AC0C93CDC4509F45BC03AC0CB3C9CE50C
:103AE000D90709F45FC0CC3CDC4509F460C030C0A4
:103AF000C23DFCE5DF0709F46FC088F4CF3C9CE5CC
:103B0000D90709F460C008F45CC0C03DFCE5DF07DC
:103B100009F45CC0C13DDC4509F45BC019C0C53D7A
:103B20009CE5D90709F460C050F4C33DFCE5DF070C
:103B300009F455C0C43DDC4509F454C009C0C63D74
:103B40009CE5D90709F455C0CE35DD4509F454C0CC
:103B500011E052C00E94691C4FC041EB5BE164EA76
:103B60007BE104C044EA5BE161EB7BE10E94171D4D
:103B700043C04AEC58E16DEB78E1F8CF4DEB58E1EA
:103B80006AEC78E1F3CF48EE58E169ED78E1EECFE9
:103B900049ED58E168EE78E1E9CF46E059E167EF99
:103BA00078E1E4CF47EF58E166E079E1DFCF49E023
:103BB00057E162EF76E1DACF42EF56E169E077E173
:103BC000D5CF81E017C065E082E010C068E086E0F4
:103BD0000DC06EE089E00AC064E18FE007C067E1D4
:103BE00085E104C088E106C062E289E10E941D1DF2
:103BF00003C083E20E94B41B812FDF91CF911F91FC
:103C00000895209A25B12E7F35B131604FB7F894D1
:103C1000FC01CB0163E070E00E94462A8E0F9F1FDB
:103C2000E817F90789F0519168E035B9000000C044
:103C300057FF25B9550F000000C000C000C025B9CE
:103C400000C06A9591F7ECCF4FBF8FE594E00197E4
:103C5000F1F700C000000895CF93DF93EC01FB0162
:103C60008281882309F43CC1C430FDE5DF0760F49C
:103C7000CB3F9CE5D90788F49E0122503C45243176
:103C8000310508F02EC109C0C236EDE5DE0729F086
:103C9000C63AFDE5DF0709F024C10E944F1090935A
:103CA0005D0280935C02C1318CE5D80709F4C6C07F
:103CB00008F042C0C930ECE5DE0709F49BC000F50E
:103CC000C5308CE5D80709F485C078F4C330ECE53D
:103CD000DE0709F478C008F07AC0C230DC4509F08C
:103CE000F5C080915C028160EFC0C7309CE5D907C8
:103CF00009F478C008F07AC080915C028061E4C069
:103D0000CD30FCE5DF0709F487C058F4CB309CE5E3
:103D1000D90709F479C008F07BC080915C02886003
:103D20006FC0CF30FCE5DF0709F480C008F082C027
:103D300080915C02877FC8C0CE3F9CE5D90709F41B
:103D400071C000F5C531FCE5DF0709F485C068F4F2
:103D5000C3319CE5D90709F475C008F095C00E94ED
:103D6000E70980915C028F77AFC0CC3FFCE5DF07AD
:103D7000A9F108F054C0CB3FDC4509F0A7C0809101
:103D80005D0240C0C230EDE5DE0709F489C058F499
:103D9000C1158DE5D80709F45AC008F069C08091B3
:103DA0005D0282602FC0C236EDE5DE0709F47CC0FB
:103DB000C63AFDE5DF0709F481C0C330DD4509F0EF
:103DC00085C080E06EC080915C0282607DC0809181
:103DD0005C0216C080915C02886076C080915D02B2
:103DE00082604FC080915C0280626EC080915C02F4
:103DF00080646AC00E94E70980915C02806864C0A8
:103E0000846062C081603DC080915C028E7F5CC036
:103E100080915C028D7F58C080915C0216C08091B9
:103E20005D0218C080915D028D7F2BC080915C0285
:103E30008F7E4AC080915C028F7D46C080915C027B
:103E40008F7B42C080915C02877F8B7F3DC08091D9
:103E50005D028D7F8E7F15C080915C0282FB2227E0
:103E600020F991E0922790FB82F990FB83F92CC016
:103E700080915D02982F909591708E7F892B90FB99
:103E800081F980935D0222C00E94E70980915C0263
:103E900087FB222720F991E0922790FB87F914C035
:103EA00081E00E94E61012C080915C0284FB222710
:103EB00020F991E0922790FB84F906C080915C0282
:103EC000982F909590FB80F980935C0280915C0222
:103ED00090915D020E9460100E94E70980E001C09D
:103EE00081E0DF91CF9108958FE891E00197F1F79C
:103EF00000C0000008950C94D70452985A9A539821
:103F00005B9A0E94741F89B182FB882780F94B99C4
:103F100002C090E001C092E0892B80932A020895AC
:103F2000E0912A02EE0FEE0FE0932A0249B142FB24
:103F3000882780F990E049B143FB222720F930E03F
:103F400043FF02C022E030E0822B932B8E2B809324
:103F50002A028F70E82FF0E0EE5AFE4F9081809198
:103F60002902890F8093290218165CF48091280297
:103F70008F5F8093280260E080E00E947B1F81E0D9
:103F800001C080E09091290297FF0AC08091280229
:103F900081508093280261E080E00E947B1F81E0D5
:103FA000109229020895CF93DF9386319C4541F505
:103FB000EB010E943F0F982F8A81209102013091DE
:103FC0000301882379F09A7A81E009F480E08093F4
:103FD0002B02911102C069E201C065E3C9010E9490
:103FE00018220AC080912B02811102C069E201C02F
:103FF00065E3C9010E9423220E94810F80E001C075
:1040000081E0DF91CF9108950F931F93CF93DF93BA
:10401000C42FD22FFC0182818823C9F040932E0245
:104020000E94DB2290932D0280932C0280E28C0F61
:10403000883008F057C0C77081E001C0880FCA956A
:10404000EAF7DF91CF911F910F910C94790780913E
:104050002E02481330C080912C0290912D020E94B4
:10406000F322883C910538F510E21D0FCD17B9F009
:1040700080E28C0F883040F4C77081E001C0880F67
:10408000CA95EAF70E948007183028F581E09D2F35
:10409000977001C0880F9A95EAF70E947907802FE0
:1040A0000E9470071830F0F4D77081E001C0880FCB
:1040B000DA95EAF70AC080E28C0F883098F4C7706E
:1040C00081E001C0880FCA95EAF7DF91CF911F9177
:1040D0000F910C948007802FDF91CF911F910F914A
:1040E0000C947007DF91CF911F910F9108950F935A
:1040F0009C01CB01243F4CE5340731F188F4293D84
:10410000FCE53F07D9F02A3D4CE5340779F1283D1D
:104110003C45A9F506E221EE41EE68ED7CE52BC0B9
:10412000263FFCE53F07E1F0A8F0273F3C4539F585
:1041300007E225EE46EE67EF7CE51DC007E225EEBF
:1041400045EE69ED7CE517C006E221EE40EE64EF36
:104150007CE511C007E225EE44EE65EF7CE50BC07F
:1041600006E221EE42EE66EF7CE505C008E221E0C2
:1041700045EE6AED7CE50E94042080E008C0FC0169
:104180008281882319F010922E0201C081E00F91E4
:10419000089590937301809372010895909334026F
:1041A000809333020895E0913302F0913402309706
:1041B00021F00190F081E02D099480E00895EF92C4
:1041C000FF921F93CF93DF93FC01A0913302B09134
:1041D0003402109709F442C080912301882341F0F2
:1041E00080915C0287FF04C08081818386E08083A8
:1041F000EF011296ED91FC911397CE0109958091F4
:10420000180282FF2BC080FF04C089E296E00E9462
:104210002E0418E083E2E82E86E0F82E8091180242
:1042200080FF0BC088811F928F93FF92EF920E94B4
:10423000C7040F900F900F900F90115021961111FD
:10424000EDCF8091180280FF09C081E296E0DF91F6
:10425000CF911F91FF90EF900C942E04DF91CF919E
:104260001F91FF90EF90089520913102309132021A
:104270002817390771F09093320280933102E09150
:104280003302F0913402309721F00680F781E02D5F
:104290000994089520912F02309130022817390790
:1042A00071F09093300280932F02E0913302F091ED
:1042B0003402309721F00084F185E02D09940895AF
:1042C000FC01329680912301882331F080915C02B9
:1042D00087FF02C09EE101C096E080E0915028F087
:1042E00021912223D9F38F5FF9CF0895662351F1ED
:1042F000209123012223E9F020915C0227FF19C0BD
:10430000462F4695469546954E31E0F4677021E07C
:1043100030E002C0220F331F6A95E2F7FC01E40F80
:10432000F11D828190E02823392381E0232B69F459
:1043300009C0FC01329608962191621729F0E8170E
:10434000F907D1F780E0089581E008959C01FC0110
:1043500032969FEF80E04191461789F09F3F19F414
:10436000411101C0982F8F5F8630A9F79F3F39F028
:10437000F901E90FF11D97FDFA95628308950895FB
:104380009C012A5F3F4FFC014281461301C012820B
:10439000019682179307B9F70895262F269526953B
:1043A00026952E3170F4FC01E20FF11D677021E0BB
:1043B00030E001C0220F6A95EAF78281282B228320
:1043C00008958091180280FF0CC01F926F9389E5B9
:1043D00096E09F938F930E94C7040F900F900F90C9
:1043E0000F900895262F2695269526952E3178F440
:1043F000FC01E20FF11D677021E030E001C0220FE7
:104400006A95EAF720958281282322830895809176
:10441000180280FF0CC01F926F938BE396E09F936E
:104420008F930E94C7040F900F900F900F900895E4
:1044300020912301222329F020915C0227FD0C9476
:10444000CD210C94A62120912301222329F0209133
:104450005C0227FD0C94F2210C94C02120912301D1
:10446000FC013296222331F080915C0287FF02C06A
:104470008EE101C086E0DF011D928A95E9F708957B
:1044800008950C94402283E0809335020C944122DD
:10449000811102C081E001C082E0809335020C945A
:1044A00041220C94482281E0809335020C944122F1
:1044B0000C94532208950C945A220C945B220C9471
:1044C0005A220C945A220C945A22CF930E946122B1
:1044D0000E94F4140E945F22C0E08C2F0E94F0130F
:1044E000811104C0CF5FC330C1F701C081E0CF911B
:1044F000089508951F920F920FB60F9211248F9373
:104500009F93AF93BF9380913602811113C0809126
:10451000750290917602A0917702B091780241964F
:10452000A11DB11D8093750290937602A09377022E
:10453000B0937802BF91AF919F918F910F900FBE72
:104540000F901F90189580917D02843031F10E9468
:10455000BE051092360220E488E190E00FB6F89490
:10456000A895809360000FBE2093600083B7817F81
:10457000846083BF83B7816083BF7894889583B755
:104580008E7F83BF0FB6F894A895809160008861F4
:1045900080936000109260000FBE08950E94E709AA
:1045A0000C94C20582E084BD93E095BD9AEF97BD5F
:1045B00080936E0008952FB7F894809175029091C2
:1045C0007602A0917702B09178022FBF08952FB79D
:1045D000F8946091750270917602809177029091C3
:1045E00078022FBF08959C014FB7F894809175020F
:1045F00090917602A0917702B09178024FBF821B12
:10460000930B089578941F920F920FB60F92112476
:104610008F939F93AF93BF93809175029091760291
:10462000A0917702B09178020196A11DB11D8093EF
:10463000750290937602A0937702B0937802BF91AF
:10464000AF919F918F910F900FBE0F901F90189573
:1046500081E08093E00080E28093D8001092C9004E
:104660008FE19EE40197F1F700C0000087E090EB36
:10467000DC018093860290938702A0938802B09316
:1046800089029CE088E10FB6F894A89580936000B9
:104690000FBE90936000FFCF80915A020895089555
:1046A0000895CF93DF9320912301222339F02091A5
:1046B0005C0227FF03C060E222E002C068E021E064
:1046C0002093E9002FEF3091E800215035FD06C01E
:1046D00035ED3A95F1F700002111F5CF2091E80072
:1046E00025FF1DC0EC0180912301811105C040E030
:1046F00050E068E070E003C070E040E050E0CE01C0
:104700000E94E1258091E8008E778093E80080E2A6
:10471000FE01AAE3B2E001900D928A95E1F7DF91E4
:10472000CF9108950895089583E896E00E942E049D
:104730000C9458228FE796E00E942E046091790233
:1047400081E0611101C080E00C9443228BE796E088
:104750000E942E0490917D0281E0943009F080E067
:10476000609179020C944822209138022F5F822FA9
:1047700062E30E94702A992319F020933802089569
:104780001092380280913902882371F180917D0264
:10479000843041F58091E9008F702091EC00922FD8
:1047A000917020FD90E8892B93E09093E90090911F
:1047B000EB0090FF14C09091EE0097FF10C0909115
:1047C000E80095FF03C01092F100F9CF9091E80046
:1047D00090FF05C09091E8009E779093E8008F705D
:1047E0008093E90010923902089542E061EC81E083
:1047F0000E94E52642E261EC82E00E94E52642E268
:1048000061EC83E00E94E52690917D0281E0943086
:1048100009F080E0609179020C94512280917F022E
:10482000833009F45DC030F4813071F0823009F4D6
:1048300096C008958A3009F482C08B3009F468C0AC
:10484000893009F0A4C020C080917E02813A09F02D
:104850009EC08091E800877F8093E800809182026B
:1048600090918302892B21F460E28AE392E003C0F5
:1048700060E080E090E070E00E942C268091E800EB
:104880008B778093E800089580917E02813209F051
:104890007EC08091820290918302029708F077C0D7
:1048A0008091E800877F8093E8008091E80082FD96
:1048B00005C080917D028111F8CF69C08091F2001E
:1048C000823031F48091F100813011F0863021F492
:1048D0008091F10080935A028091E8008B7753C059
:1048E00080917E02813A09F052C0809182029091BB
:1048F0008302892B09F04BC08091E800877F809369
:10490000E8008091E80080FFFCCF8091230136C051
:1049100080917E028132D9F580918202909183024A
:10492000892BA9F58091E800877F8093E8000E9499
:104930001A2780918002809323010C94E7098091CB
:104940007E02813221F58091E800877F8093E80024
:104950000E941A278091810280935B0208958091C2
:104960007E02813AA1F48091E800877F8093E8007D
:104970008091E80080FFFCCF80915B028093F10082
:104980008091E8008E778093E8000C941A270895B0
:104990009FB7F894109239029FBF90917D02943096
:1049A00009F057C09091E9009F703091EC00232FDF
:1049B000217030FD20E8922B23E02093E900209124
:1049C000EB0020FF43C02091EE0027FF3FC0209165
:1049D0003702222321F02091E80025FF37C01092F2
:1049E000370226E03091E80035FD15C030917D0298
:1049F000343061F53091EB0035FD28C0215021F4B1
:104A000081E08093370222C0EFE9FFE03197F1F7B0
:104A100000C00000E7CF8093F1008091E80085FDA1
:104A20000AC08091E80080FFFCCF8091E8008E777B
:104A30008093E80006C08FB7F89421E020933902F4
:104A40008FBF9F709093E90080E008959F709093CE
:104A5000E9008FEF089584B7877F84BF0FB6F8947D
:104A6000A89580916000886180936000109260003A
:104A70000FBE90E080E80FB6F894809361009093A9
:104A800061000FBE0C9453220E946C270E94BF2726
:104A9000E2EEF0E080818460808378940C94222A96
:104AA00087E191E00C94CE2080917D028530C9F49D
:104AB00087E796E00E942E0480917D02853079F48C
:104AC0000E94A32280917B028823B1F30E94652279
:104AD000882391F30E94CB250E94E709EDCF0C9427
:104AE000CE22089508950C947525292F332723305D
:104AF0003105C9F060F42130310581F022303105F3
:104B000009F041C08BE590E025EC36E040C0213251
:104B10003105E1F02232310531F135C082E190E01A
:104B200020E237E034C099278130910549F028F020
:104B3000029749F5E7E8F6E005C0E1ECF6E002C0CF
:104B4000E9E9F6E0849190E09F0121C063307105AE
:104B5000D0F4660F771FFB01E559FE4F20813181AC
:104B600089E090E014C06330710568F4FB01EE0F3A
:104B7000FF1FEB59FE4F20813181FB01EE59FE4FA3
:104B8000808190E004C080E090E020E030E0FA0115
:104B900031832083089584E089BD86E089BD09B40E
:104BA00000FEFDCF8091D8008F7D8093D80080914A
:104BB000E00082608093E0008091E00081FDFCCF06
:104BC0000895CF92DF92EF92FF920F931F93CF93AE
:104BD000DF93EC018B017A010E943927811133C0E8
:104BE000E114F10439F0F70180819181081B190B60
:104BF000C80FD91FC12CD12C0115110519F18091B5
:104C0000E80085FD16C08091E8008E778093E8006B
:104C1000E114F10449F0F70180819181C80ED91E99
:104C2000D182C08285E00FC00E943927882321F3FA
:104C30000AC089918093F10001501109FFEFCF1A4A
:104C4000DF0ADACF80E0DF91CF911F910F91FF90C3
:104C5000EF90DF90CF9008952091840230918502EB
:104C60002617370748F06115710539F42091E800DF
:104C70002E772093E80001C0B901FC0120E0611506
:104C8000710561F180917D028823D9F18530D9F1D8
:104C90008091E80083FD39C08091E80082FD2BC03F
:104CA0008091E80080FFEBCF8091F20090E06115E9
:104CB000710551F08830910538F421912093F1006D
:104CC000615071090196F3CF21E0089709F020E0C7
:104CD0008091E8008E778093E800D1CF2111D2CF68
:104CE0000AC080917D02882361F0853061F0809157
:104CF000E80083FD0AC08091E80082FFF2CF80E0E7
:104D0000089582E0089583E0089581E00895209158
:104D10008402309185022617370748F06115710526
:104D200039F42091E8002E772093E80001C0B90102
:104D3000FC0120E06115710579F180917D028823E5
:104D400009F43DC0853009F43CC08091E80083FD42
:104D50003AC08091E80082FD2CC08091E80080FF7D
:104D6000E9CF8091F20090E06115710559F088302B
:104D7000910540F424912093F1003196615071091E
:104D80000196F2CF21E0089709F020E08091E80039
:104D90008E778093E800CECF2111CFCF0AC08091CB
:104DA0007D02882361F0853061F08091E80083FD09
:104DB0000AC08091E80082FFF2CF80E0089582E08F
:104DC000089583E0089581E00895982F953068F55F
:104DD0009093E900981739F07091EC002091ED0064
:104DE0005091F00003C0242F762F50E021FD02C027
:104DF0009F5FECCF3091EB003E7F3093EB00309122
:104E0000ED003D7F3093ED003091EB003160309349
:104E1000EB007093EC002093ED005093F000209194
:104E2000EE0027FDE5CF80E008958F708093E900C4
:104E300081E0089580917E0287FF11C08091E80093
:104E400082FD05C080917D028111F8CF11C0809153
:104E5000E8008B770BC080917D02882349F0809118
:104E6000E80080FFF8CF8091E8008E778093E8001B
:104E700008952091E4003091E50095E64091EC0022
:104E8000842F817040FF23C08091E80080FD1DC009
:104E900080917D02882399F0853099F08091EB0014
:104EA00085FD11C04091E4005091E50024173507BD
:104EB00029F3915011F09A01E1CF84E0089582E046
:104EC000089583E0089581E0089580E00895409179
:104ED000E80042FFDDCF08950E94C9270E94CC2739
:104EE000E0EEF0E0808181608083E8EDF0E0808199
:104EF0008F77808319BCE3E6F0E080818160808356
:104F000010927C0208950E94C9270E94CC278091AC
:104F1000D8008F778093D8008091D80080688093E4
:104F2000D8008091D8008F7D8093D80084E089BD1F
:104F300086E089BD09B400FEFDCF10927D0210927B
:104F4000790210927B0210927A0242E060E080E0E7
:104F50000E94E5268091E1008E7F8093E1008091A0
:104F6000E20081608093E2008091E200886080939B
:104F7000E2008091E0008E7F8093E0000895E3E6F8
:104F8000F0E080818E7F808381E080937C020C94AE
:104F900083271092E20008951092E10008951F9275
:104FA0000F920FB60F9211242F933F934F935F935D
:104FB0006F937F938F939F93AF93BF93EF93FF93E1
:104FC0008091E10082FF0BC08091E20082FF07C068
:104FD0008091E1008B7F8093E1000E94B423809157
:104FE000E10080FF19C08091E20080FF15C0809130
:104FF000E2008E7F8093E2008091E20080618093E6
:10500000E2008091D80080628093D80019BC85E0CE
:1050100080937D020E949A238091E10084FF30C03A
:105020008091E20084FF2CC084E089BD86E089BDC8
:1050300009B400FEFDCF8091D8008F7D8093D80009
:105040008091E1008F7E8093E1008091E2008F7E6D
:105050008093E2008091E20081608093E200809181
:105060007902882311F084E007C08091E30087FD76
:1050700002C081E001C083E080937D020E94A623EC
:105080008091E10083FF29C08091E20083FF25C069
:105090008091E100877F8093E10082E080937D0230
:1050A000109279028091E1008E7F8093E1008091DF
:1050B000E2008E7F8093E2008091E2008061809325
:1050C000E20042E060E080E00E94E5268091F0008E
:1050D00088608093F0000E949423FF91EF91BF912C
:1050E000AF919F918F917F916F915F914F913F9180
:1050F0002F910F900FBE0F901F9018951F920F9237
:105100000FB60F9211242F933F934F935F936F939A
:105110007F938F939F93AF93BF93CF93DF93EF933F
:10512000FF93C091E900CF708091EC00D82FD1702F
:1051300080FDD0E81092E9008091F000877F809395
:10514000F00078940E94C2281092E9008091F0004B
:1051500088608093F000CD2BCF70C093E900FF9161
:10516000EF91DF91CF91BF91AF919F918F917F91FF
:105170006F915F914F913F912F910F900FBE0F90C4
:105180001F9018951F93CF93DF93CDB7DEB7AA97E3
:105190000FB6F894DEBF0FBECDBFEEE7F2E0809110
:1051A000F100819322E0E638F207C9F70E940E244D
:1051B0008091E80083FF2EC180917E0290917F0252
:1051C000492F50E04A30510508F024C1FA01EA5B4A
:1051D000FF4F0C94C62A803821F0823809F01AC19A
:1051E00008C080917A0290917B02992389F08260B5
:1051F0000FC0809182028F70853008F00BC18093C0
:10520000E9008091EB0085FB882780F91092E90086
:105210009091E800977F9093E8008093F1001092BE
:10522000F100D1C0282F2D7F09F0F4C0882319F098
:10523000823061F0EFC080918002813009F0EAC0D5
:10524000933009F080E080937B022EC08091800231
:1052500081112AC0809182028F702FEF280F243095
:1052600008F0D8C08093E9002091EB0020FF1CC01B
:10527000933021F48091EB00806214C09091EB0098
:1052800090619093EB0021E030E0A90102C0440F4F
:10529000551F8A95E2F74093EA001092EA00809148
:1052A000EB0088608093EB001092E9008091E800A9
:1052B000877F8093E8000E941A27ACC08111AAC0A2
:1052C000109180021F778091E3008078812B80937A
:1052D000E3008091E800877F8093E8000E941A270E
:1052E0008091E80080FFFCCF8091E300806880938C
:1052F000E300111102C082E001C083E080937D02CF
:1053000089C08058823008F085C0809180029091D9
:1053100081028C3D53E0950779F583E08A838AE228
:1053200089834FB7F894DE01139620E03EE051E206
:10533000E32FF0E050935700E49120FF03C0E29583
:10534000EF703F5FEF708E2F90E0EA3010F0C7965D
:1053500001C0C0968D939D932F5F243149F74FBFB5
:105360008091E800877F8093E8006AE270E0CE01D8
:1053700001960E942C2616C06091820270918302D1
:10538000AE014F5F5F4F0E947325BC01892B09F46A
:1053900041C09091E800977F9093E80089819A81BD
:1053A0000E9487268091E8008B778093E80032C0C6
:1053B000803881F58091E800877F8093E8008091B4
:1053C00079028093F1008091E8008E7772CF81118D
:1053D00021C0809180029091810299270297D4F494
:1053E0008091E800877F8093E8008091800280931D
:1053F00079020E941A2780917902811106C080915A
:10540000E30087FD02C081E001C084E080937D025B
:105410000E94F5238091E80083FF0AC08091E80094
:10542000877F8093E8008091EB0080628093EB009F
:10543000AA960FB6F894DEBF0FBECDBFDF91CF9115
:105440001F910895CF9380917D028823A1F0C09190
:10545000E900CF709091EC00892F817090FD80E879
:10546000C82B1092E9008091E80083FD0E94C228B9
:10547000CF70C093E900CF910895002480FD060EFF
:10548000660F11F08695D1F7802D089500245527D9
:1054900004C0080E591F880F991F009729F07695B0
:1054A0006795B8F37105B9F7802D952F0895EE270C
:1054B000FF27AA27BB2708C0A20FB31FE41FF51FB1
:1054C000220F331F441F551F969587957795679533
:1054D00098F37040A9F7009799F7BD01CF0108959F
:1054E000991B79E004C0991F961708F0961B881F36
:1054F0007A95C9F780950895AA1BBB1B51E107C097
:10550000AA1FBB1FA617B70710F0A61BB70B881F53
:10551000991F5A95A9F780959095BC01CD010895E2
:1055200097FB072E16F4009407D077FD09D00E9450
:105530007C2A07FC05D03EF4909581959F4F0895F5
:10554000709561957F4F0895A1E21A2EAA1BBB1B8F
:10555000FD010DC0AA1FBB1FEE1FFF1FA217B3073F
:10556000E407F50720F0A21BB30BE40BF50B661F55
:10557000771F881F991F1A9469F760957095809519
:1055800090959B01AC01BD01CF010895EE0FFF1F67
:105590000590F491E02D0994FC014150504030F009
:1055A00001900616D1F73197CF01089588279927E2
:1055B0000895FB01DC0104C08D910190801921F454
:1055C00041505040C8F7881B990B0895F999FECFB8
:1055D00092BD81BDF89A992780B50895A6E1B0E003
:1055E00044E050E00C94202BA8E1B0E042E050E011
:1055F0000C94202B262FF999FECF92BD81BDF89AED
:10560000019700B4021639F01FBA20BD0FB6F89406
:10561000FA9AF99A0FBE08950396272F0E94FB2A43
:105620000E94FA2A252F0E94FB2A242F0C94FB2A81
:105630000196272F0E94FB2A0C94FA2ADC01CB0149
:10564000FC01F999FECF06C0F2BDE1BDF89A319692
:1056500000B40D9241505040B8F70895F894FFCF30
:10566000C800E701010102000400040401191A1B2B
:105670001C1D1E1F2021224C235123922393234FB4
:105680002350230134353637679064659100010259
:105690000202020606060909090909090F0F0F0F80
:1056A0000F0F15151518191919191919191919198B
:1056B000232400FF0100010000FFFF0000010001A2
:1056C000FF00403B228F0754073207D706F0060938
:0256D0000700D1
:00000001FF
